:020000040800F2
:10000000B0040020010100086F1500081711000856
:100010006D150008990100084D1800080000000047
:10002000000000000000000000000000DB150008D8
:100030003502000800000000D9150008DD15000891
:100040001B0100081B0100081B0100081B01000820
:100050001B0100081B0100081B0100081B01000810
:100060001B0100081B0100081B0100081B01000800
:100070001B0100081B0100081B0100081B010008F0
:100080001B0100081B0100081B0100081B010008E0
:100090001B0100081B0100081B0100081B010008D0
:1000A0001B0100081B0100081B0100081B010008C0
:1000B0001B0100081B0100081B0100081B010008B0
:1000C0001B0100081B0100081B0100081B010008A0
:1000D0001B0100081B0100081B0100081B01000890
:1000E0001B0100081B0100081B010008DFF80CD0F1
:1000F00000F040F800480047FD190008B004002057
:100100000648804706480047FEE7FEE7FEE7FEE7B1
:10011000FEE7FEE7FEE7FEE7FEE7FEE73116000832
:10012000ED000008D2B201E000F8012B491EFBD21D
:1001300070470022F6E710B513460A4604461946F2
:10014000FFF7F0FF204610BD30B50B4601460020FA
:100150002022012409E021FA02F59D4205D303FA89
:1001600002F5491B04FA02F52844151EA2F101020A
:10017000F1DC30BD064C074D06E0E06840F00103BD
:1001800094E8070098471034AC42F6D3FFF7B2FF6B
:10019000C81B0008E81B0008FEE700001FB510237D
:1001A0008DF80C00012203A98DE80E0013460246CB
:1001B00004480188044800F0D5F99DF80C0004B00B
:1001C00010BD000000000020180000201FB5002115
:1001D00003911023022203A98DE80E000246054870
:1001E00001230188044800F0BDF9BDF80C0004B0FB
:1001F00010BD000000000020180000201FB50022E4
:1002000003928DF80C101023012203A98DE80E0033
:100210001346024602480188024800F0B3FA1FBDA7
:1002200000000020180000200149088070470000ED
:10023000000000207047704770B5044600F0ECF8ED
:100240000546601C02D004480078044400F0E4F83D
:10025000401BA042FAD370BD040000202DE9F84FE6
:10026000DFF890A100220AF1040B144601274FF099
:100270000F090BF1040E00BF0B6807FA04F52B40C1
:10028000AB4274D1DFF870C14E68A6EB0C0866452E
:100290002BD00DDC032E34D005DC36B3012E19D063
:1002A000022E2FD11BE0112E16D0122E2AD119E0CA
:1002B000B8F5881F19D006DCB8F5803F15D0B8F521
:1002C000801F1FD111E0B8F5001F0ED0B8F5041F34
:1002D00018D10AE0CA6815E0CA68121D12E0CA689F
:1002E00008320FE0CA680C320CE08A682AB1012A91
:1002F0004FF0080203D0456104E0042202E00561EA
:1003000000E00022FF2B01D8064601E000F10406C0
:100310004FEA840501D9A5F12005D6F800C009FAF5
:1003200005F82CEA080C02FA05F54CEA050CC6F8AB
:1003300000C04D68ED0057D5304DAE6946F001065E
:10034000AE61AD6924F0030605F0010500952C4D62
:1003500006EB050CDCF80850A6074FEA167809FAF8
:1003600008F6B543274EB04202D1002610E03BE02C
:10037000254EB04201D101260AE0244EB04201D1FF
:10038000022605E0224EB04201D1032600E00426F9
:1003900006FA08F62E43CCF808604D68DAF80060DB
:1003A000ED03554601D51E4300E09E432E604D6887
:1003B000DBF80060AD035D4601D51E4300E09E43BF
:1003C0002E604D68DEF80060ED02754601D51E43D3
:1003D00000E09E432E604D68AD020E4D2E6801D5A3
:1003E0001E4300E09E432E60641C102CFFF444AFBB
:1003F000BDE8F88F00040140000011100010024019
:100400000000014000080140000C014000100140C4
:10041000001401400C04014001488068704700004E
:100420000400002070B504001BD094F83D000025A6
:1004300020B984F83C50204600F042FA242084F889
:100440003D002068016821F00101016000F0B0FB6F
:10045000404A6168914201D83F4900E03F498842E3
:1004600001D2012070BD3E492368B0FBF1F1596013
:100470006368934206D94FF4967359434FF47A73E5
:10048000B1FBF3F12368491C19626168914210D8ED
:100490004900401EB0FBF1F2521CC2F30B02042AC9
:1004A00001D2042022E0B0FBF1F0401CC0F30B00AD
:1004B0001CE0A368CBB301EBC10202EB0116421EA4
:1004C000B2FBF6F2521C42F48042120536D06BB3F6
:1004D00001EBC10202EB0111401EB0FBF1F0401C28
:1004E000C0F30B0040F4804040F400402168C86134
:1004F000D4E90701084321680860D4E903100843E0
:1005000021688860D4E9050108432168C860206833
:10051000016841F0010101602564202084F83D005C
:10052000256384F83E50002070BD00E008E001EB38
:100530004106421EB2FBF6F2521CC6E70120D5E787
:1005400001EB4101401EB0FBF1F0401CC0F30B0079
:10055000CAE70000A086010080841E0000093D005B
:1005600040420F002DE9FF4F83B09A46DDE9118725
:1005700093460446DDF84090FFF74EFF054694F899
:100580003D00202872D1192301227B492046009585
:1005900000F0C5FE0028F5D194F83C00012865D094
:1005A000012084F83C0020680168C90703D1016874
:1005B00041F0010101602068016821F400610160DF
:1005C000222084F83D00402084F83E000026266466
:1005D000C4F82490A4F82A806848E062608D2085E1
:1005E000CDE9007553465A462046049900F0A8FD0F
:1005F00028B1206C84F83C60042851D075E0208D2F
:10060000DFF87C8168B1012814D0022820680168D5
:100610001ED041F4806101602068416980690090CA
:100620009BE02068416981690091016841F4007193
:10063000016092E02068016821F48061016072B677
:100640002068416981690091016841F400710AE004
:1006500041F40061016072B62068416981690091CE
:10066000016821F48061016062B676E081E00328D0
:1006700050D801280BD002283B464FF000024146DB
:100680002046009512D000F04AFE70BB13E02A46C7
:100690003946204600F0B8FE30B1206C202824D026
:1006A000012007B0BDE8F08F20684BE000F037FE76
:1006B000D8B972B61BE02068016821F4806101603E
:1006C00072B620680169606A421C62620170208D06
:1006D000401E2085608D401E60853B4600224146BD
:1006E0002046009500F01BFE08B10320D9E72068E2
:1006F000016841F40071016020680169606A421C70
:1007000062620170208D401E2085608D401E6085D4
:1007100062B6C9E72A463946204600F075FE002831
:10072000BBD120680169606A421C62620170208D41
:10073000401E2085608D401E608520684169C94348
:1007400049070AD40169606A421C62620170208D07
:10075000401E2085608D401E6085208D002886D13A
:10076000202084F83D0084F83E6084F83C6000203E
:1007700097E7022095E70000020010000000FFFF4D
:10078000040001002DE9FF4F83B09A46DDE911878F
:1007900093460446DDF84090FFF73EFE064694F887
:1007A0003D0020287DD1192301224349204600968F
:1007B00000F0B5FD00287CD194F83C00012878D0E9
:1007C000012084F83C0020680168C90703D1016852
:1007D00041F0010101602068016821F400610160BD
:1007E000212084F83D00402084F83E000025256447
:1007F000C4F82490A4F82A803048E062608D2085F7
:10080000CDE9007653465A462046049900F010FD83
:1008100080B3206C84F83C50042848D008E032466D
:100820003946204600F021FE30B1206C042839D032
:10083000032007B0BDE8F08F606A411C6162216847
:1008400000780861208D401E80B22085618D491E90
:10085000618521684A69D24352070BD468B1606A46
:10086000421C626200780861208D401E2085608DE8
:10087000401E6085208D0028D1D132463946204661
:1008800000F026FD0028D0D154F83D0B016841F45A
:1008900000710160202004F81E09E57765770020CB
:1008A000C7E706E02068016841F40071016001209B
:1008B000BFE70220BDE70000020010000000FFFFBC
:1008C00010B586B00021009101910291039100685A
:1008D0001349884222D1134CA06940F00800A0615E
:1008E000A069694600F0080004904FF44070009041
:1008F00012200190032003900B48FFF7AFFC0B4838
:10090000416841F0E06141F002014160E06940F47A
:100910000010E061E06900F40010049006B010BD22
:100920000054004000100240000C01400000014053
:1009300002488168027811448160704704000020F9
:10094000074810B5016841F010010160032000F074
:1009500067F8002000F006F800F024F8002010BD31
:100960000020024070B50D4D04464FF47A7128788E
:10097000B1FBF0F00A490968B1FBF0F000F0F0FAC1
:1009800048B9102C07D200222146501E00F028F84A
:1009900000206C6070BD012070BD000004000020CC
:1009A000100000200C4808B5816941F00101816107
:1009B000816901F001010091C16941F08051C1617B
:1009C000C06900F0805000900448416821F0E06167
:1009D00041F00071416008BD00100240000001407C
:1009E000F0B40E4B1B680C46C3F30223C3F107059A
:1009F000042D00D90425191D072901D2002300E088
:100A0000DB1E012606FA05F1491E214099409E4051
:100A1000761E16403143F0BC00F0AABD0CED00E09C
:100A2000064900F0070208684FF6FF03184040EA45
:100A30000220034A10430860704700000CED00E0FC
:100A40000000FA052DE9F047DFF8548105460E460F
:100A5000D8F8000000F00700B0420CD2D8F800101F
:100A600021F007013143C8F80010D8F8000000F069
:100A70000700B0426FD128684A4C810712D5400761
:100A800003D5606840F4E06060602878000703D513
:100A9000606840F4605060606068A96820F0F00011
:100AA000084360602878C00744D06868012816D0E1
:100AB0002168022816D0890700294CDA616821F0E4
:100AC000030101436160FFF7A7FC6968074641F233
:100AD000883001290ED00229814618D026E02168ED
:100AE0008903E9E78901E7E7FFF796FCC11B494560
:100AF00001D918E081466068C0F381000128F3D174
:100B000018E000BFFFF788FCC11B49450BD860689F
:100B1000C0F381000228F5D10CE000BFFFF77CFC98
:100B2000C11B494502D90320BDE8F087606810F079
:100B30000C0FF3D1D8F80010404601F00701B14284
:100B40000BD9016821F0070131430160006800F012
:100B50000700B04201D00120E6E72878400705D51C
:100B60006068E96820F4E060084360602878000766
:100B700006D56068296920F4605040EAC1006060D1
:100B800000F036F86168084AC1F30311515CC840AF
:100B9000064908600020FFF7E5FE0020C4E70000DA
:100BA0000020024000100240B01B0008100000208E
:100BB0000448054900684968044AC1F30221515CB0
:100BC000C84070471000002000100240C01B000801
:100BD0000448054900684968044AC1F3C221515CD0
:100BE000C84070471000002000100240C01B0008E1
:100BF00012A185B00FC98DE80F0014A0144A006837
:100C000004905168134801F00C03042B10D0082BFA
:100C10000ED1C1F38343C9031DF803000AD55168FF
:100C200004AAC1F34041515C0A4A5043B0FBF1F0C1
:100C300005B0704708494843FAE70000020304057D
:100C4000060708090A0B0C0D0E0F10100102000018
:100C50000010024000127A0000093D002DE9F84F13
:100C600004460078B94DC00748D06868C0F38100D9
:100C7000012807D06868C0F38100022809D168689C
:100C8000C00306D52868800338D5606800286FD077
:100C900034E06068B0F5803F0BD010B1B0F5A02F04
:100CA00011D0286820F480302860286820F4802043
:100CB00002E0286840F480302860606888B1FFF75F
:100CC000ABFB064609E0286840F480202860F0E786
:100CD000FFF7A2FB801B642875D828688003F7D52E
:100CE0000CE0FFF799FB064605E000BFFFF794FB19
:100CF000801B6428F0D828688003F7D42078944EAD
:100D000080074FF001094FF000083BD5686810F0EC
:100D10000C0F07D06868C0F38100022809D1686809
:100D2000C00306D42868800714D5206901281FD184
:100D300010E02069B0B1C6F80090FFF76DFB0746E0
:100D400005E000BFFFF768FBC01B0228C4D8286875
:100D50008007F7D52868616920F0F80040EAC100F3
:100D600028600FE0C6F80080FFF756FB074606E054
:100D7000E9E000BFFFF750FBC01B022823D828681A
:100D80008007F7D4207800072CD57248A169D9B123
:100D9000C0F80090FFF740FB074604E0FFF73CFB7C
:100DA000C01B02280FD8686A8007F7D56A484FF43D
:100DB000FA510068B0FBF1F0009000BF0098411EAE
:100DC0000091FAD20EE080E0C0F80080FFF724FB2B
:100DD000074604E0FFF720FBC01B022875D8686AAD
:100DE0008007F7D42078400760D5E8690027C00065
:100DF00008D4E86940F08050E861E869012700F014
:100E00008050009055480168C90513D40168834695
:100E100041F480710160FFF7FFFA824606E000BFEF
:100E2000FFF7FAFAA0EB0A0064284ED8DBF80000BE
:100E3000C005F5D5E06801280AD008B1052813D00F
:100E4000286A20F001002862286A20F0040002E0ED
:100E5000286A40F001002862E06841F2883B98B1BE
:100E6000FFF7DAFA82460BE0286A40F004002862B5
:100E7000EEE700BFFFF7D0FAA0EB0A0159455AD8B8
:100E8000286A8007F6D50CE0FFF7C6FA824605E02F
:100E9000FFF7C2FAA0EB0A0159454CD8286A80072F
:100EA000F6D41FB1E86920F08050E861E06988B3AA
:100EB0006968C1F38101022945D00228C6F8608023
:100EC00004D0FFF7A9FA044638E034E0FFF7A4FAAB
:100ED000074604E0FFF7A0FAC01B02282BD82868B9
:100EE0008001F7D4206AB0F5803F05D16868A16819
:100EF00020F4003008436860D4E9080108436968B9
:100F000021F4741108436860C6F86090FFF784FA12
:100F1000044606E015E000BFFFF77EFA001B02283A
:100F200009D828688001F7D50BE000BFFFF774FAF5
:100F3000001B022802D90320BDE8F88F2868800131
:100F4000F4D40020F8E70120F6E70000001002408A
:100F50000000424280044242100000200070004025
:100F600010B5401EB0F1807F01D3012010BD4FF0BD
:100F7000E02460610F21601700F0FAFA0020A06100
:100F800007202061002010BD70B5040004D094F843
:100F90003900002510B106E0012070BD84F83850FA
:100FA000204600F023F8242084F839002068C16826
:100FB00021F40051C160204600F05EFB2068016909
:100FC00021F4904101612068416921F02A014161C9
:100FD0002068C16841F40051C160E563202084F8B5
:100FE000390084F83A00002070BD000030B585B0AB
:100FF00000240094019402940394006814498842E8
:1010000023D11448C16941F40031C161C16901F4BF
:1010100000310491816941F00401816180690E4DC4
:1010200000F00400049004200090022001900320AE
:10103000039069462846FFF711F90820CDE900041E
:10104000694628460294FFF709F905B030BD000053
:101050000044004000100240000801402DE9F84320
:10106000044690F839001F4616460D46202850D1F8
:10107000A5B19EB194F8380001284AD0012084F827
:1010800038004FF00008C4F83C80212084F8390073
:10109000FFF7C2F9A6848146E68426E00120BDE878
:1010A000F883E08C401EE084A0684B46B0F5805F7A
:1010B0004FF000024FF080012046009703D000F06F
:1010C00093FBE8B90DE000F08FFBC8B928882168D0
:1010D000C0F308004860206908B16D1C05E0AD1C34
:1010E00003E0216815F8010B4860E08C0028D8D196
:1010F0004B46002240212046009700F075FB08B1C6
:101100000320CCE7202084F8390084F838800020C0
:10111000C5E70220C3E7FEE701684A69D2435205EA
:101120000CD46FF480624A6104210164002140F80C
:10113000301F202242730173012070470020704746
:101140002DE9F84F0446006889460B9D01689846D2
:10115000174641F4806101602068016841F48071A4
:10116000016000954FF0011A0022514620460A9B6B
:1011700000F0D5F8F0BB216809F0FE0008610AF123
:10118000010B2B46594620460A9A00F0F9F818B18F
:10119000206C042812D03AE02068416980690090F0
:1011A0002A4620460A9900F060F950B1206C0428C4
:1011B0002DD12068016841F4007101600120BDE873
:1011C000F88FFEB2B8F1010F09D02168380A086122
:1011D0002A4620460A9900F048F90028E6D12068FE
:1011E00006612A4620460A9900F03FF90028DDD121
:1011F000206800E00BE0016841F480710160009517
:101200000022514620460A9B00F089F808B10320CD
:10121000D5E7216809F0FF0040F0010008612B4686
:10122000594620460A9A00F0ABF80028B0D1C6E72C
:101230002DE9F843044600680D46DDE9089701688A
:101240009846164641F4807101604B4600224FF0EB
:1012500001112046009700F062F8E8B9216805F016
:10126000FE0008613B464A461849204600F088F8CF
:1012700028B1206C04280FD10120BDE8F883206834
:101280004169806900903A464946204600F0EDF8F1
:1012900020B1206C042813D00320EEE7F5B2B8F19A
:1012A000010F09D02168300A08613A4649462046B4
:1012B00000F0DBF80028ECD1206805610020DCE7B5
:1012C0002068016841F400710160D5E70200010067
:1012D00070B516460D4604461AE02046FFF71CFF7F
:1012E00008B1012070BD681C12D025B1FFF794F839
:1012F000801BA8420CD954F8400F40F0200044F85D
:10130000100900202060202161732073032070BD2C
:1013100020684069C0434007DFD4002070BD2DE93C
:10132000F0471E4690460D460446C1F30747DDF8D8
:10133000209012E0701C10D02EB1FFF76DF8A0EBDA
:101340000900B04209D9002044F8300F2021617310
:10135000A07320730320BDE8F0872068012F0AD016
:10136000806925EA00000004000C06D000214145F8
:10137000E0D00020EFE74069F3E70121F7E7000044
:101380002DE9F0479A4691460D46044600264FF057
:101390002008C1F307472AE020684069C0434005A0
:1013A00012D42068016841F40071016021686FF473
:1013B0008060486104202064266384F83D8084F8BE
:1013C0003C600120BDE8F087B9F1FF3F0FD0B9F1D3
:1013D000000F05D0FFF720F8A0EB0A01494506D918
:1013E00044F8306F84F80D8026730320EAE7206804
:1013F000012F07D0D0F8180025EA00000004000CE7
:10140000E0D0C9E74069F7E72DE9F04100259046B3
:101410000E460446202721E04069C043C0060CD494
:1014200021686FF0100048612564256384F83D70E1
:1014300084F83C500120BDE8F0812EB1FEF7ECFFAE
:10144000A0EB0800B04209D954F8400F40F020004A
:1014500044F80409677025700320ECE720684169AF
:10146000C9434906D8D40020E5E770B516460D46B5
:1014700004461AE02046FFF74FFE08B1012070BD78
:10148000681C12D025B1FEF7C7FF801BA8420CD9FB
:1014900054F8400F40F0200044F81009002020606C
:1014A000202161732073032070BD20684069C04310
:1014B0000006DFD4002070BD0D4808B5816941F0F9
:1014C00020018161816901F020010091816941F071
:1014D00004018161816901F004010091816941F099
:1014E00008018161806900F00800009008BD0000DB
:1014F000001002400D4810B50B4901600C494160D5
:1015000000214FF480428160C0E903124161816192
:10151000C1610162FEF786FF002803D0BDE81040DC
:10152000FEF789BE10BD00000054004018000020E6
:10153000A08601000C4810B50A4901604FF4E13162
:101540004160002181600C22C160C0E90412816108
:10155000C161FFF719FD002803D0BDE81040FEF778
:101560006ABE10BD004400406C000020FEE77047DA
:101570000907090E002806DA00F00F0000F1E0204C
:1015800080F8141D704700F1E02080F800147047C7
:1015900070B5E620FEF748FE0520FEF74DFE002060
:1015A000FEF7FCFD202801D0002070BD0021EF20B7
:1015B000FEF724FE074D002405EB4400417815F8A2
:1015C0001400FEF71BFE641CE4B2332CF4D301209C
:1015D00070BD0000041B000870477047FFF7A8B9F2
:1015E00030B58FB028216846FEF7A3FD14210AA864
:1015F000FEF79FFD01210804CDE9001000240294AC
:1016000002250491CDE907504FF4E0100990684697
:10161000FFF724FB0F20CDE90A056802CDE90C4055
:1016200002210AA80E94FFF70DFA0FB030BD00009A
:101630000D48016841F00101016041680B4A114009
:10164000416001680A4A11400160016821F480216B
:101650000160416821F4FE0141604FF41F01816087
:101660000449C00308607047001002400000FFF802
:10167000FFFFF6FE08ED00E02DE9F04104460068AA
:101680000169E26821F44051114301612169A068B8
:101690000843616908432168CA6841F20C639A43B0
:1016A0000243CA6020684169A26921F44071114374
:1016B00041614C4920686425322688423CD1FFF7BD
:1016C00087FA00EBC00101EB001061688900B0FBF4
:1016D000F1F7FFF77DFA00EBC00101EB0010616844
:1016E000B0468900B0FBF1F0B0FBF5F06FF01801E7
:1016F000484307EB800106EB0110B0FBF5F000F06A
:10170000F006FFF765FA00EBC00101EB001061681D
:101710008900B0FBF1F0B0FBF5F006EB0016FFF727
:1017200057FA00EBC00101EB001061688900B0FBC3
:10173000F1F7FFF74DFA3BE0FFF73AFA00EBC00193
:1017400001EB001061688900B0FBF1F7FFF730FA98
:1017500000EBC00101EB00106168B0468900B0FBEE
:10176000F1F0B0FBF5F06FF01801484307EB800192
:1017700006EB0110B0FBF5F000F0F006FFF718FAE9
:1017800000EBC00101EB001061688900B0FBF1F0D3
:10179000B0FBF5F006EB0016FFF70AFA00EBC0010C
:1017A00001EB001061688900B0FBF1F7FFF700FA68
:1017B00000EBC00101EB001061688900B0FBF1F0A3
:1017C000B0FBF5F06FF01801484307EB800108EB20
:1017D0000110B0FBF5F0216800F00F003044886084
:1017E000BDE8F081003801402DE9F04198461746E8
:1017F0000E460446069D1DE0681C1BD02DB1FEF769
:101800000BFEA0EB0800A84214D92068C16821F49F
:10181000D071C1602068416921F00101416120203F
:1018200084F8390084F83A00002084F83800032056
:10183000BDE8F0812068006836EA000004D000208E
:10184000B842D9D00020F3E70120F9E7FEE7000015
:101850000FB4054B10B503A9044A029800F018F81C
:1018600010BC5DF814FB0000E5190008140000200E
:1018700002E008C8121F08C1002AFAD17047704759
:10188000002001E001C1121F002AFBD170470000B7
:101890002DE9FF4F89B09B460446002506E0252828
:1018A0000BD05A460B999047641C6D1C2078002879
:1018B000F5D10DB02846BDE8F08F0027B8460122CB
:1018C000474900E0074314F8013F203B02FA03F0C8
:1018D0000842F7D120782E2819D114F8010F47F0CB
:1018E00004072A280ED06FF02F022078A0F13001D3
:1018F00009290CD808EB880102EB410100EB010833
:10190000641CF2E70A98641C50F8048B0A90207853
:101910000028CED0642808D0692806D075281ED0AB
:101920005A460B9990476D1C58E00A994FF00A09E6
:1019300001C90A91002802DA40422D2102E039054E
:1019400004D52B218DF82010012103E0F90704D0E4
:101950002021F7E78A4608AE0DE00021FAE70A9950
:101960004FF00A0901C90A91F7E74946FEF7ECFB77
:10197000303106F8011D0028F7D1ADEB060000F16B
:101980002009780701D44FF00108C84502DDA8EB13
:10199000090000E000208046002706E008A85A461B
:1019A000C05D0B9990476D1C7F1C5745F6DB04E02A
:1019B00030205A460B9990476D1CB8F10001A8F1F0
:1019C0000108F5DC05E016F8010B5A460B99904723
:1019D0006D1CB9F10001A9F10109F4DC641C65E793
:1019E0000928010013B54FF6FF730122694602482A
:1019F000FFF734FB00981CBD6C00002070B5FEF7AB
:101A00009FFFFFF7EDFDFFF757FDFFF793FDFFF792
:101A100071FD1BA0FFF71CFFFFF7BAFD00282AD0BD
:101A200020A0FFF715FF0021EF20FEF7E7FB234D75
:101A3000002400BF05EB4400417815F81400FEF7C0
:101A4000DDFB641CE4B2232CF4D30021EF20FEF76D
:101A5000D5FB4FF49675B020FEF7A0FB0446B120ED
:101A6000FEF7B4FB0246214615A0FFF7F1FE28461B
:101A7000FEF7E2FBEFE71DA0FFF7EAFE002070BDD6
:101A8000476573747572652053656E736F72205469
:101A90006573742050726F6772616D202E2E2E0D4B
:101AA0000A0000000A476573747572652053656EFD
:101AB000736F72204F4B0D0A000000006A1B000874
:101AC0004F626A656374206272696768746E6573D9
:101AD00073203D202564202C4F626A656374207357
:101AE000697A65203D2025640D0A00000A47657368
:101AF000747572652053656E736F72204572726FD4
:101B0000720D0A00EF00370738173906410042000E
:101B1000462D470F483C49004A1E4C2051105E108C
:101B200060278042814482048B019006950A960CBE
:101B300097059A149C3FA519CC19CD0BCE13CF64F1
:101B4000D021EF01020F0310040225012739287F5D
:101B500029083EFF5E3D6596679769CD6A016D2C49
:101B60006E017201733574007701EF00410042008D
:101B7000483C49005113832084208500861087004B
:101B8000880589188A109FF869966A02EF01011E7C
:101B9000020F031004024150433465CE660B67CE3A
:101BA000680B69E96A056B506CC36D506EC37405B0
:101BB00000000000000000000102030406070809FD
:101BC0000000000001020304E81B000800000020E0
:101BD0001800000070180008001C00081800002001
:101BE0009804000080180008E600000001000000D2
:101BF000100000000000000000A24A0400000000E5
:04000005080000ED02
:00000001FF
